:020000040000FA
:1008000064EF1DF01200FFFFFFD71200FFFFFFFF94
:10081000FFFFFFFFFFFFFFFF3CEF19F01200FFFF9C
:10082000FFFFFFFFFFFFFFFFFFFF0400F73A00009D
:10083000C400000002000000F63A0000CA000000F8
:1008400001000000F43A0000C200000002000000B5
:10085000F13A0000C900000001000000E30E8A1612
:10086000F30E931693886BEC1AF037EF04F04D0EED
:10087000E66E010EE66E6C0EE66E12EC1CF0E552B2
:10088000E552E552130E146E2B0E156E166A14C047
:10089000E6FF15C0E6FF16C0E6FF79EC1CF0E55256
:1008A000E552E5520001C96BD7EF11F0060E0001C9
:1008B000BC5D03E36D50020B01E001D001D81200D2
:1008C000D9CFE6FFE1CFD9FF050EE126040EDB6AA2
:1008D000400EE66E620EE66E000EE66E2BEC1AF02F
:1008E000E552E552E552000902E144EF0AF0000149
:1008F000C90538E10E0E146E2B0E156E166A14C063
:10090000E6FF15C0E6FF16C0E6FF10EC1BF0E5524F
:10091000E552E552010EDB6A100EF36E010EDBCFDD
:10092000F4FFF350F45C1EE2010EDB50EA6A620F42
:10093000E96E000EEA22EF50E66EE66A0A0E146EC9
:100940002B0E156E166A14C0E6FF15C0E6FF16C022
:10095000E6FF10EC1BF0F56E050EE15EF550010EA2
:10096000DB2ADAD70001606B400E0001625D02E015
:10097000EBEF09F000016351FF0A02E1D7EF09F044
:10098000A90A02E1A7EF09F0140A02E172EF09F0E7
:100990000E0A02E146EF09F00D0A02E116EF09F036
:1009A000060A01E1E5D3010A01E194D3170A01E146
:1009B00037D3150A01E1EDD2160A01E1A3D2020AEA
:1009C00001E14FD2070A01E1E9D1030A01E194D123
:1009D000070A01E13DD1100A01E10FD10D0A01E141
:1009E000E1D04D0A01E1ACD0070A01E17DD0060A51
:1009F00058E04D0A3EE04E0A20E0010A02E0D9EF3D
:100A000009F0030EE66E4AEC0AF0E55200090EE02A
:100A10000001646B0001030E656F040EE66E88EC46
:100A20000AF0E5520001050E606F05D00B0EF36E63
:100A3000040EF3CFDBFFEAEF09F0030EE66E4AEC9B
:100A40000AF0E55200090EE00001646B0001010E9E
:100A5000656F040EE66E88EC0AF0E5520001050EA3
:100A6000606F05D00B0EF36E040EF3CFDBFFEAEFE1
:100A700009F0030EE66E4AEC0AF0E55200090AE0BE
:100A80008A76020EE66E88EC0AF0E5520001030E4B
:100A9000606F05D00B0EF36E040EF3CFDBFFEAEFB1
:100AA00009F0040EE66E4AEC0AF0E552000915E082
:100AB000020E64C0DBFF020EDB5004E00001010EF9
:100AC000C96F02D00001C96B020EE66E88EC0AF015
:100AD000E5520001030E606F05D00B0EF36E040E9D
:100AE000F3CFDBFFEAEF09F0030EE66E4AEC0AF003
:100AF000E55200090BE0D9EC19F0020EE66E88EC25
:100B00000AF0E5520001030E606F05D00B0EF36E84
:100B1000040EF3CFDBFF0001C90510E1EC0E146EEB
:100B20002A0E156E166A14C0E6FF15C0E6FF16C041
:100B3000E6FF10EC1BF0E552E552E552EAEF09F052
:100B4000030EE66E4AEC0AF0E552000911E0D5EC1E
:100B500019F00001646FD1EC19F00001656F040E0B
:100B6000E66E88EC0AF0E5520001050E606F05D0D4
:100B70000B0EF36E040EF3CFDBFF0001C90510E18D
:100B8000CF0E146E2A0E156E166A14C0E6FF15C03D
:100B9000E6FF16C0E6FF10EC1BF0E552E552E55209
:100BA000EAEF09F0030EE66E4AEC0AF0E55200099E
:100BB0000BE0D7EC11F0020EE66E88EC0AF0E5527D
:100BC0000001030E606F05D00B0EF36E040EF3CF21
:100BD000DBFF0001C90510E1B60E146E2A0E156E7A
:100BE000166A14C0E6FF15C0E6FF16C0E6FF10EC5B
:100BF0001BF0E552E552E552EDD3030EE66E4AECEA
:100C00000AF0E55200090BE0FFEC11F0020EE66E6F
:100C100088EC0AF0E5520001030E606F05D00B0E60
:100C2000F36E040EF3CFDBFF0001C90510E19C0E4B
:100C3000146E2A0E156E166A14C0E6FF15C0E6FF84
:100C400016C0E6FF10EC1BF0E552E552E552C2D3A8
:100C5000030EE66E4AEC0AF0E552000934E001ECBE
:100C600012F0E76E030EE7CFDBFF030EDB5009E166
:100C7000020EE66E88EC0AF0E5520001030E606F8A
:100C800021D00001C90510E17A0E146E2A0E156EEE
:100C9000166A14C0E6FF15C0E6FF16C0E6FF10ECAA
:100CA0001BF0E552E552E5520001650E636F030E3D
:100CB000DBCF64F0030EE66E88EC0AF0E55200012B
:100CC000040E606F05D00B0EF36E040EF3CFDBFF46
:100CD0000001C90510E1600E146E2A0E156E166A29
:100CE00014C0E6FF15C0E6FF16C0E6FF10EC1BF0CF
:100CF000E552E552E5526ED3030EE66ECBDBE552CC
:100D0000000933E039EC12F0E76E030EE7CFDBFFAA
:100D1000030EDB5009E1020EE66E88EC0AF0E552A4
:100D20000001030E606F20D00001C90510E13F0EE5
:100D3000146E2A0E156E166A14C0E6FF15C0E6FF83
:100D400016C0E6FF10EC1BF0E552E552E55200013B
:100D5000650E636F030EDBCF64F0030EE66ED8DB27
:100D6000E5520001040E606F05D00B0EF36E040E09
:100D7000F3CFDBFF0001C90510E1260E146E2A0E29
:100D8000156E166A14C0E6FF15C0E6FF16C0E6FF32
:100D900010EC1BF0E552E552E5521CD3020E64C084
:100DA000DBFF040EE66E76DBE552000935E064C039
:100DB000E6FFADEC12F0E552E76E030EE7CFDBFF86
:100DC000030EDB5008E1020EE66EA2DBE5520001E5
:100DD000030E606F20D00001C90510E10F0E146EE4
:100DE0002A0E156E166A14C0E6FF15C0E6FF16C07F
:100DF000E6FF10EC1BF0E552E552E5520001650EEE
:100E0000636F030EDBCF64F0030EE66E81DBE55209
:100E10000001040E606F05D00B0EF36E040EF3CFCD
:100E2000DBFF0001C9051CE1030EDBCFE6FFE66A2C
:100E3000C550E66EE66A020EDBCFE6FFE66AD70E25
:100E4000146E290E156E166A14C0E6FF15C0E6FF73
:100E500016C0E6FF10EC1BF0F56E090EE15EF550D2
:100E6000B9D2030EE66E16DBE552000932E071ECF2
:100E700012F0E76E030EE7CFDBFF030EDB5008E155
:100E8000020EE66E45DBE5520001030E606F20D0D6
:100E90000001C90510E1B00E146E290E156E166A18
:100EA00014C0E6FF15C0E6FF16C0E6FF10EC1BF00D
:100EB000E552E552E5520001650E636F030EDBCF8C
:100EC00064F0030EE66E24DBE5520001040E606F51
:100ED00005D00B0EF36E040EF3CFDBFF0001C90546
:100EE00010E1930E146E290E156E166A14C0E6FFFB
:100EF00015C0E6FF16C0E6FF10EC1BF0E552E55208
:100F0000E55268D2030EE66EC5DAE552000923E029
:100F1000D950020FE66E000EDA20E66EE8EC12F011
:100F2000E552E552E76E030EE7CFDBFF030EDB5021
:100F300004E1020EDBCF64F006D00001650E636FA2
:100F4000030EDBCF64F0030EE66EE2DAE552000139
:100F5000040E606F05D00B0EF36E040EF3CFDBFFB3
:100F60000001C90515E100016451E66EE66A710EE3
:100F7000146E290E156E166A14C0E6FF15C0E6FF42
:100F800016C0E6FF10EC1BF0F56E050EE15EF550A5
:100F900021D2030EE66E7EDAE552000923E0D95035
:100FA000020FE66E000EDA20E66ECCEC12F0E5528F
:100FB000E552E76E030EE7CFDBFF030EDB5004E1E3
:100FC000020EDBCF64F006D00001650E636F030EE6
:100FD000DBCF64F0030EE66E9BDAE5520001040EEF
:100FE000606F05D00B0EF36E040EF3CFDBFF000134
:100FF000C90515E100016451E66EE66A4C0E146EF7
:10100000290E156E166A14C0E6FF15C0E6FF16C05D
:10101000E6FF10EC1BF0F56E050EE15EF550DAD13F
:10102000020E64C0DBFF020EDB50040FE66E32DA04
:10103000E552000931E0020EDB50200805E2200EE7
:10104000F36E020EF3CFDBFF64C0E6FF650EE66EC3
:10105000000EE66E86EC13F0E552E552E552E76EBF
:10106000030EE7CFDBFF030EDB5008E1020EE66E56
:101070004FDAE5520001030E606F0DD00001650EDE
:10108000636F030EDBCF64F0030EE66E41DAE552C8
:101090000001040E606F05D00B0EF36E040EF3CF4B
:1010A000DBFF0001C90515E1020EDBCFE6FFE66AB2
:1010B0002B0E146E290E156E166A14C0E6FF15C0AD
:1010C000E6FF16C0E6FF10EC1BF0F56E050EE15EC4
:1010D000F55080D1080EE66EDDD9E552000942E0F8
:1010E000020E68C0DBFF020EDB50200805E2200E76
:1010F000F36E020EF3CFDBFF640EE66E000EE66EBB
:10110000020EDBCFE6FF67C0E6FF66C0E6FF65C004
:10111000E6FF64C0E6FF04EC13F0F56E070EE15E37
:10112000F550E76E030EE7CFDBFF030EDB500CE15B
:10113000020EDB50020FE66EEBD9E552020EDB50D9
:10114000030F0001606F0DD00001650E636F030E89
:10115000DBCF64F0030EE66EDBD9E5520001040E2E
:10116000606F05D00B0EF36E040EF3CFDBFF32D1B0
:10117000040EE66E8FD9E552000939E0020E64C014
:10118000DBFF020EDB50200805E2200EF36E020E9C
:10119000F3CFDBFF020EDBCFE6FF640EE66E000E40
:1011A000E66E68EC13F0E552E552E552E76E030E89
:1011B000E7CFDBFF030EDB500CE1020EDB50020F2A
:1011C000E66EA6D9E552020EDB50030F0001606FF8
:1011D0000DD00001650E636F030EDBCF64F0030ECC
:1011E000E66E96D9E5520001040E606F05D00B0E35
:1011F000F36E040EF3CFDBFF0001C90516E1020E0A
:10120000DB50020FE66EE66A080E146E290E156EAC
:10121000166A14C0E6FF15C0E6FF16C0E6FF10EC24
:101220001BF0F56E050EE15EF550D4D0030EE66EB0
:1012300031D9E55200090CE008EC14F00001646FAC
:10124000030EE66E65D9E5520001040E606F05D00D
:101250000B0EF36E040EF3CFDBFF0001C90515E1A1
:1012600000016451E66EE66AE30E146E280E156EF8
:10127000166A14C0E6FF15C0E6FF16C0E6FF10ECC4
:101280001BF0F56E050EE15EF550A4D0040EE66E7F
:1012900001D9E55200090DE064C0E6FFF9EC13F056
:1012A000E552020EE66E34D9E5520001030E606F7E
:1012B00005D00B0EF36E040EF3CFDBFF0001C90562
:1012C00010E1C50E146E280E156E166A14C0E6FFE6
:1012D00015C0E6FF16C0E6FF10EC1BF0E552E55224
:1012E000E55278D0040EE66ED5D8E552000911E03B
:1012F000020E64C0DBFF020EDBCFE6FFE6EC11F06E
:10130000E552020EE66E04D9E5520001030E606F4D
:1013100005D00B0EF36E040EF3CFDBFF0001C90501
:1013200015E1020EDBCFE6FFE66AA10E146E280E71
:10133000156E166A14C0E6FF15C0E6FF16C0E6FF7C
:1013400010EC1BF0F56E050EE15EF55043D0030E78
:10135000E66EA0D8E55200090CE0FCEC11F00001AB
:10136000646F030EE66ED4D8E5520001040E606F80
:1013700005D00B0EF36E040EF3CFDBFF0001C905A1
:1013800015E100016451E66EE66A7D0E146E280ECA
:10139000156E166A14C0E6FF15C0E6FF16C0E6FF1C
:1013A00010EC1BF0F56E050EE15EF55013D0FF005A
:1013B00011D00001040E606F0001400E626F000149
:1013C000650E636F00010A0E646F030EE66EA0D80F
:1013D000E55200D010D00001040E606F0001400EF5
:1013E000626F0001650E636F00010C0E646F030EE7
:1013F000E66E8ED8E552040EDB500DE00001650E5E
:10140000636F040EDBCF64F0030EE66E81D8E55205
:101410000001040E606F0001605123E004010CBF65
:101420000CD060C0E6FF620EE66E000EE66EF1ECD8
:1014300019F0E552E552E55213D00001C90510E15B
:10144000650E146E280E156E166A14C0E6FF15C0E0
:10145000E6FF16C0E6FF10EC1BF0E552E552E55240
:1014600013D00001C90510E1480E146E280E156E48
:10147000166A14C0E6FF15C0E6FF16C0E6FF10ECC2
:101480001BF0E552E552E552D9CFE1FFE552E7CF37
:10149000D9FF1200D9CFE6FFE1CFD9FF020EE12636
:1014A000010E62C0DBFFDF6EFE0EDB50DF5C10E280
:1014B000DF50EA6A620FE96E000EEA22010EDBCF0E
:1014C000E7FFEF50E71A010EE7CFDBFFDF2AECD78B
:1014D000010EDB5002E1010E15D00001C90510E13B
:1014E000300E146E280E156E166A14C0E6FF15C075
:1014F000E6FF16C0E6FF10EC1BF0E552E552E552A0
:10150000000E00D0D9CFE1FFE552E7CFD9FF12009E
:10151000D9CFE6FFE1CFD9FF020EE126010E62C06E
:10152000DBFFDF6EFE0EDB50DF5C10E2DF50EA6AAD
:10153000620FE96E000EEA22010EDBCFE7FFEF50EB
:10154000E71A010EE7CFDBFFDF2AECD7FE0EDB50F8
:10155000EA6A620FE96E000EEA22010EDBCFEFFFAE
:10156000D9CFE1FFE552E7CFD9FF1200F2EC0FF03F
:10157000FB0EDBCFF3FFDB06F35000090AE040EC83
:1015800010F0FA0EABEC10F0F3E1151CF1E1010ED6
:1015900001D0000E21EF10F0F2EC0FF03B0EE12431
:1015A00002E3E168E652E16E010EDB6A020EDB6ADD
:1015B000F90EDBCFF6FFFA0EDBCFF7FFFB0EDBCF2A
:1015C000F8FF0800F550DF6EDF5002E147EF0FF043
:1015D000250EDF5C02E03AEF0FF0030EDB6A040E2B
:1015E000DB6A050EDB6A060EDB6A070EDB6A5AEC65
:1015F0000FF02D0EDF5C0CE02B0EDF5C09E0200EFF
:10160000DF5C06E0230EDF5C03E0300EDF5C1AE1F6
:10161000DF50300A14E0130A0FE0030A0AE00B0A55
:1016200005E0060AE4E1030EDB80E1D7030EDB826E
:10163000DED7030EDB84DBD7030EDB86D8D7030EA1
:10164000DB88D5D72A0EDF5C1BE156EC0FF0A4EC4B
:101650000FF010E0030EDB8006680768130EDBCF87
:101660000BF0140EDBCF0CF0ABEC1CF0040E04C03E
:10167000DBFF03D0130E8DEC0FF05AEC0FF00BD004
:10168000090EDB6AFBEC0FF003E06FEC10F0FAD709
:10169000090E8DEC0FF0030EDBB0DB982E0EDF5C35
:1016A0001BE15AEC0FF02A0EDF5C0BE156EC0FF059
:1016B000A4EC0FF003E1130EDFEC0FF05AEC0FF087
:1016C0000BD0090EDB6AFBEC0FF003E06FEC10F0BF
:1016D000FAD7090EDFEC0FF0680EDF5C07E15AEC79
:1016E0000FF0680EDF5C1DE1030E18D0740EDF5C96
:1016F00017E07A0EDF5C14E0480EDF5C06E0540E63
:10170000DF5C03E05A0EDF5C02E1020E07D06C0ED4
:10171000DF5C03E06A0EDF5C04E1010E32EC10F0E6
:10172000C9DBDF506E0A01E181D31E0A01E192D1CB
:10173000200A01E18FD13F0A01E149D11A0A01E1F2
:1017400046D10D0A01E143D1200A01E140D13A0A14
:1017500001E13DD1200A01E13AD1260A01E135D16A
:101760000D0A01E132D11A0A01E1D9D0200A4AE07A
:10177000300A1FE0460A0EE0250A01E085D3D95061
:10178000F90FE96EFF0EDA20EA6E010EEE5E000E32
:10179000EE5AEE5A40EC10F0250EE66E95DB03E1B2
:1017A000151C01E16BD33CEC10F001E26DD3DB2A98
:1017B0006BD3080EDB6A040EDB50010806E2040E50
:1017C000DB0404EC10F0DB508BDB080EDB5009E08F
:1017D000030EDB50010B05E172DB01E04FD3080E75
:1017E000DB6A64DBEFCFDFFFB4EC10F003E1151C24
:1017F00001E144D33CEC10F001E3DB2A60DB01E1C2
:1018000043D33CD3070EDB5002080FE180EC10F00D
:10181000030E47EC10F00E0EEECFDBFF0F0EEECFF7
:10182000DBFF100EEECFDBFF20D0F70EDBCF17F083
:10183000F80EDBCF18F0020E175E000E185AF70EE6
:1018400017C0DBFFF80E18C0DBFF17C0E9FF18C098
:10185000EAFF37EC10F0166A0E0E14C0DBFF0F0E15
:1018600015C0DBFF100E16C0DBFF0E0EDBCFE6FF50
:101870000F0EDBCFE6FF100EDBCFE6FF54EC1CF0C3
:10188000E552E552E552130E05C0DBFF140E06C00B
:10189000DBFF060EDB5005E0130E7BEC10F001E2DF
:1018A0006ADB9FEC10F002E2130E37DB62EC10F003
:1018B00006E0040E7BEC10F002E2050E2EDB030EB8
:1018C000DBB005D0FCDA01E0D9D2080EDB6A090EE4
:1018D000DB6A0E0EDBCFF6FF0F0EDBCFF7FF100E2D
:1018E000DBCFF8FF0800F550DF6EDF5014E0A5EC09
:1018F00010F011E2B4EC10F003E1151C01E1BED2CE
:10190000BBDB01E3DB2A090EDB2AD9500E0FE96E9F
:10191000000ECBDBE7D7D3DA01E1B6D2AFD2C6DA1D
:10192000110EEECFDBFF120EEDCFDBFF110EDBCF82
:10193000E6FF120EDBCFE6FF46EC1CF0E552E55267
:10194000130EF3CFDBFF140EF4CFDBFF060EDB50DC
:1019500004E0130ED0DB01E20EDB9FEC10F002E29C
:10196000130EDBDAAFDB05E0040EC5DB02E2050E89
:10197000D4DA030EDBB005D0A2DA01E07FD2080E84
:10198000DB6A090EDB6A110EDBCFE9FF120EDBCF3B
:10199000EAFFEFCFDFFFDF5014E0D7DB12E2E4DB3A
:1019A00003E1151C01E16AD267DB01E3DB2A090EC2
:1019B000DB2A110EDB2ADBCFE9FF120EE8E3DB2A7C
:1019C000E6D77DDA01E160D259D2030EDB8E070E35
:1019D000DB0410E195DB040E5ADB0A0EEECFDBFFD1
:1019E0000B0EEECFDBFF0C0EEECFDBFF0D0EEECFBE
:1019F000DBFF6CD0070EDB5003082CE1030EDBAEDF
:101A00000DD0B2DA020E76DAEFCF14F0156A166A4C
:101A1000176A14AE39D01568166835D0F70EDBCFCB
:101A200015F0F80EDBCF16F0020E155E000E165AFA
:101A3000F70E15C0DBFFF80E16C0DBFF15C0E9FF7F
:101A400016C0EAFFEFCF14F00A0E14C0DBFF0B0E36
:101A5000DB6A38D0070EDB50020809E1030EDBAE6B
:101A600004D059DB16AE10D00ED055DB0DD0030ECE
:101A7000DBAE12D079DA020E3DDAF9DA166A176AAD
:101A800015AE02D016681768E2DA0C0E16C0DBFF3E
:101A90000D0E17C0DBFF1AD0F70EDBCF16F0F80ED5
:101AA000DBCF17F0020E165E000E175AF70E16C0A7
:101AB000DBFFF80E17C0DBFF16C0E9FF17C0EAFF17
:101AC000D6DAC5DA0C0EDB6A0D0EDB6A060EDB50C9
:101AD00005E1010EF36E050EF3CFDBFF150EDB6A99
:101AE000160EDB6AD950370F146E000EDA20156E11
:101AF000390E14C0DBFF3A0E15C0DBFF380EDB6A6F
:101B0000080EDB6A0A0EAEDADF50780A12E0200A0D
:101B100010E0280A0CE0200A0AE03F0A06E00D0A5D
:101B200002E0200A08E1020E05D0080E03D0080EDC
:101B3000DF26100E97DA030EDBBE02D0DB92DB94B9
:101B4000DB50800B26E08ADA030EEB50000AE8AE89
:101B500002D0D89008D0000EEE5C000EEE58000EB9
:101B6000EE58000EEE5815E211DA09680A680B68A3
:101B70000C68DAEC1BF00A0E00C0DBFF0B0E01C094
:101B8000DBFF0C0E02C0DBFF0D0E03C0DBFF2D0ED2
:101B900008D0030EDBA202D02B0E03D0DBA408D0AA
:101BA000200EF36E170EF3CFDBFF150EDB2A02D0EB
:101BB000170EDB6A050EDB5003E1B5D901E189D0D0
:101BC000E00E146E3A0E156E000E166E070EDBCF89
:101BD00017F0186A196A1A6A17C009F018C00AF0D3
:101BE00019C00BF01AC00CF0D1D9D8EC1CF014506D
:101BF0000024F36E15500120F46E16500220F86E8A
:101C0000F4CFF7FFF3CFF6FF0800090EF5CFDBFFA7
:101C1000580EDF5C0FE1610EF36E090E79D90AE30D
:101C2000200E146E090EDBCFE7FF1450E75E090E9D
:101C3000E7CFDBFF070EDBCF14F0156A166A176AD1
:101C40000DDA14C009F015C00AF016C00BF017C069
:101C50000CF0EECF04F0EECF05F0EECF06F0EFCFB4
:101C600007F0D8EC1CF007C0EDFF06C0EDFF05C083
:101C7000EDFF04C0EFFF390EDBCFE9FFDB063A0EC4
:101C8000DBCFEAFF01E2DB06090EDBCFEFFF150E2B
:101C9000DB2A49D995E1030EDBA61DD06F0EDF5C70
:101CA00006E1BFD918E3150EDB2859DA14D0780EF7
:101CB000DF5C09E0580EDF5C06E0620EDF5C03E0EB
:101CC000420EDF5C08E1020EF36E160EF3CFDBFF6F
:101CD00002D0150EDB6A030EDB50100B0EE0040E73
:101CE000DBCF14F0050EDB50D880145406E2060E4C
:101CF000DB5003E1040EDB5032DA93D90AE2050E21
:101D0000DBCFE7FF150EDB50E75E050EE7CFDBFF0D
:101D100002D0050EDB6A040EDBCF14F0160E43D999
:101D2000D880145414E2160EDBCFE6FF150EDBCF7D
:101D3000E6FF040EDBCFE6FF050EDB50E552E75C65
:101D4000E552D880E754E552D880E7545DD9030EB8
:101D5000DB50010B0BE1080EDB5008E0B0D801E0CE
:101D60008DD0080EDB50BCD8080EDB6A170EDB5096
:101D700007E086D9170EEFD903E1151C01E17ED0EB
:101D8000160EDB5016E07CD9300EE66E9DD802E1CF
:101D9000151C74E075D9DFCFE6FF5AEC1BF0E55255
:101DA000E552E552F4CF15F00001F31C02E1151CD9
:101DB00065E0050EDBCF14F0160EDB50D88014540E
:101DC00009E2050EDBCFE7FF160EDB50E75E050EDE
:101DD000E7CFDBFF300EE66E050EC9D94FE1390EB5
:101DE000DB2ADBCFE9FF3A0E01E3DB2ADBCFEAFF98
:101DF000090EEFCFDBFFDB500EE042D9090EABD965
:101E000002E1151C3BE0390EDB2ADBCFE9FF3A0E7D
:101E1000EDE3DB2AEBD753D831E1160EDBCFE6FF3B
:101E2000080EC1D8E552E7245BD82ED0070EDB5050
:101E3000030A1CE0010A14E0030A07E079D9DBCFAA
:101E4000EEFF020EDBCFEDFF1FD0F3D8196A17AEFD
:101E500002D0186819682AD8BAD819C0EEFF14D071
:101E6000E8D817BE186822D8B2D80ED061D9DBCF17
:101E7000EFFF0AD079D905E1151C03E1F368F46896
:101E800010D0FAD801E3DB2A77D9E1EF0AF0010E8E
:101E9000DBCF14F0020EDBCF15F014C0F3FF15C03A
:101EA000F4FFD9CFE1FFDACFE2FFCBD029D9020E80
:101EB00047EF10F061D90800F550DF6E1200200ED8
:101EC000E66E080EB7EF10F05AEC1BF0E552E55243
:101ED000E552F3CF14F0F4CF15F00001F31C12001B
:101EE000146E156AD950010F4DD91450EE261550B5
:101EF000ED221200185E000E195AF70E18C0DBFF13
:101F0000F80E19C0DBFF18C0E9FF19C0EAFF120084
:101F1000DBCFF4FFF350F45C1200DB50E76E040EED
:101F2000E7CFDBFF12000A0EDBCF14F00B0EDBCF86
:101F300015F00C0EDBCF16F00D0EDBCF17F01450A2
:101F40001510161017101200130EEECFDBFF140E33
:101F5000EDCFDBFF130EDBCF14F0140EDBCF15F04B
:101F60000001800E15141200F70EDBCF18F0F80EEA
:101F7000DBCF19F01200050EDB50E66ED950130FBF
:101F800001D9E552E750EE6EED6A12000A0EDBCF82
:101F900004F00B0EDBCF05F00C0EDBCF06F00D0EC0
:101FA000DBCF07F01200DBCFE6FF150EDBCFE6FF3D
:101FB000050EDB50E552E724E552E7241200DB5022
:101FC000CED8010EF36E060EF3CFDBFF1200EE50FB
:101FD000EFCFEAFFE96E16C0EEFF17C0EEFF18C0A4
:101FE000EEFF1200D9CFE6FFDACFE6FFE1CFD9FF4F
:101FF000E2CFDAFF1200DFCFE6FFE66A44EC1DF025
:10200000E552E552F3501200E76E080EE7CFDBFF12
:102010001200EECF14F0EECF15F0EFCF16F0176AE6
:102020001200050EDBCF14F0150EDB50D8801454CF
:102030001200010EDBCF16F0020EDBCF17F0186A8C
:102040001200E552E5CFDAFFE7CFD9FF12000A0E02
:1020500014C0DBFF0B0E15C0DBFF1200D9500A0FB6
:10206000C2EF10F0F36E070EF3CFDBFF1200EECFDE
:1020700014F0EFCF15F01200010EDB2A020E120051
:10208000FC0EDBCFE6FFFD0EDBCFE6FF1200145E99
:10209000000E155AF70E14C0DBFFF80E15C0DBFF5B
:1020A00014C0E9FF15C0EAFF1200DA20EA6EEF2A39
:1020B000EECFF6FF000EEF22EECFF7FFEF22EECFCE
:1020C000F8FF1200040EDBCFE6FF130EDB50E552E3
:1020D000E75C9ADFDB5004DF060EDB501200090ECE
:1020E000DB500A0DF350DF24D00FE76E090EE7CF67
:1020F000DBFF5AEF0FF0DB50F36E050E88EF0FF0A9
:10210000F70EDBCF14F0F80EDBCF15F01200DFCFA7
:10211000E6FF64EF0FF028DF030EECDE09EF10F0AE
:10212000B6EC0AF0E552E552E552E552000912001C
:10213000BDDEEE50EFCFEAFFE96E010E1200130E86
:10214000DB50F36E040E88EF0FF0040EDB50F36EDD
:10215000090E88EF0FF0DBCFE6FF64EF0FF0E76EBC
:10216000050EE7CFDBFF12008BDF87EF10F0DBCF30
:10217000E6FF86DF90EF10F0D950F90FE96EFF0E01
:1021800055EF10F0E96E000EDA20EA6E1200D9CF9A
:10219000E6FFE1CFD9FF020EE126DE68DD68C586E5
:1021A000D9CFE9FFDACFEAFFEE06000EED5AEECF07
:1021B00014F0EDCF15F01450151006E0C7A003D0B1
:1021C000C596010E04D0ECD7C596000E00D0D9CF2D
:1021D000E1FFE552E7CFD9FF1200C95000D012004D
:1021E000D9CFE6FFE1CFD9FF020EE126DE68DD6838
:1021F000A196FE0EDB50C96EDE68DD68040EC714C2
:1022000010E0D9CFE9FFDACFEAFFEE06000EED5A73
:10221000EECF14F0EDCF15F01450151002E00400CD
:10222000EDD7D9CFE9FFDACFEAFFEE50ED1003E1A9
:1022300020D90D0E30D0A1A603D0A196030E2BD02D
:10224000C6AE04D0C69E020E26D015D0DE68DD686C
:10225000C750010B10E0D9CFE9FFDACFEAFFEE0655
:10226000000EED5AEECF14F0EDCF15F0145015100E
:1022700002E00400EDD7A1A603D0A196030E0BD077
:10228000D9CFE9FFDACFEAFFEE50ED1002E1060EFA
:1022900002D0000E00D0D9CFE1FFE552E7CFD9FF41
:1022A0001200D9CFE6FFE1CFD9FF020EE126DE68AA
:1022B000DD68A196FC0EDBCFF3FFDB06F3500009CF
:1022C00049E0040064DF00090FE087DFE66EFD0EE1
:1022D000DBCFE9FFDB2AFE0EDBCFEAFF01E3DB2ADF
:1022E000E552E750EF6E02D0010E5BD0A1A603D0FD
:1022F000A196030E56D0FC0EDB502BE0A196C59A9A
:10230000C588DE68DD68C550100B15E0D9CFE9FF40
:10231000DACFEAFFEE06000EED5AEECF14F0EDCF65
:1023200015F01450151007E00400A1A603D0A196E3
:10233000030E37D0E8D7D9CFE9FFDACFEAFFEE5066
:10234000ED1002E1050E2DD0A1A603D0A196030E3B
:1023500028D0B0D7C58AC588DE68DD68C550100BA7
:1023600015E0D9CFE9FFDACFEAFFEE06000EED5A0D
:10237000EECF14F0EDCF15F01450151007E0040067
:10238000A1A603D0A196030E0CD0E8D7D9CFE9FFC0
:10239000DACFEAFFEE50ED1002E1050E02D0000E9A
:1023A00000D0D9CFE1FFE552E7CFD9FF1200E66AAE
:1023B000080EE66EFCEC1CF0E552E552F18EC78C7F
:1023C0001D0EE66E03D8E552A1961200D9CFE6FFA6
:1023D000E1CFD9FFC69AE66A080EE66EFCEC1CF067
:1023E000E552E552C586F18EC78CFE0EDB50C86EF5
:1023F000E552E7CFD9FF1200C85000D01200C69AAC
:102400001200D9CFE6FFE1CFD9FF020EE126DE6848
:10241000DD68A196C580010EC51415E0D9CFE9FF8E
:10242000DACFEAFFEE06000EED5AEECF14F0EDCF54
:1024300015F01450151007E00400A1A603D0A196D2
:10244000030E11D0E8D7A1A603D0A196030E0BD09E
:10245000D9CFE9FFDACFEAFFEE50ED1002E1070E27
:1024600002D0000E00D0D9CFE1FFE552E7CFD9FF6F
:102470001200D9CFE6FFE1CFD9FF020EE126DE68D8
:10248000DD68A196C584A1A603D0A196030E23D032
:10249000040EC51410E0D9CFE9FFDACFEAFFEE064B
:1024A000000EED5AEECF14F0EDCF15F014501510CC
:1024B00002E00400EDD7A1A603D0A196030E0BD035
:1024C000D9CFE9FFDACFEAFFEE50ED1002E1080EB6
:1024D00002D0000E00D0D9CFE1FFE552E7CFD9FFFF
:1024E0001200D9CFE6FFE1CFD9FF020EE126DE6868
:1024F000DD68C582A1A603D0A196030E28D0020EE6
:10250000C51415E0D9CFE9FFDACFEAFFEE06000ED9
:10251000ED5AEECF14F0EDCF15F01450151007E082
:102520000400A1A603D0A196030E11D0E8D7D9CFFD
:10253000E9FFDACFEAFFEE50ED1002E1090E07D015
:10254000A1A603D0A196030E02D0000E00D0D9CFD1
:10255000E1FFE552E7CFD9FF1200D9CFE6FFE1CF87
:10256000D9FFE652FE0EDBCFE6FF3ADEE552DF6E24
:10257000A1A603D0A196030E0AD0DF5002E0DF50DF
:1025800006D0C5AC02D0040E02D0000E00D0E55239
:10259000E552E7CFD9FF1200D9CFE6FFE1CFD9FF4F
:1025A000F6DD00090FE019DEE66EFD0EDBCFE9FF78
:1025B000FE0EDBCFEAFFE552E750EF6EC58AC58815
:1025C000000E02D0010E00D0E552E7CFD9FF120075
:1025D000D9CFE6FFE1CFD9FFDADD00090FE0FDDD5D
:1025E000E66EFD0EDBCFE9FFFE0EDBCFEAFFE55224
:1025F000E750EF6EC59AC588000E02D0010E00D0DC
:10260000E552E7CFD9FF1200D9CFE6FFE1CFD9FFDE
:10261000E652F7DEDF6EDF5002E0DF5054D0FD0EF1
:10262000DB50E824E66E99DFE552DF6EDF5002E012
:10263000DF5049D0FE0EDB5007E1FB0EDBCFE6FF9B
:102640008CDFE552DF6E13D0FE0EDB0410E1FC0ED2
:10265000DBCFE6FF82DFE552DF6EDF5002E0DF50C6
:1026600032D0FB0EDBCFE6FF78DFE552DF6EDF50C6
:1026700002E0DF5028D035DFDF6EDF5002E0DF50B0
:1026800022D0FD0EDB50E8240109E66E66DFE5523C
:10269000DF6EDF5002E0DF5016D00400FA0EDBCF11
:1026A000E6FFF80EDBCFE6FFF90EDBCFE6FF10D832
:1026B000E552E552E552DF6EDF5002E0DF5003D015
:1026C000D8DE000E00D0E552E552E7CFD9FF120068
:1026D000D9CFE6FFE1CFD9FFE652FC0EDBCFE6FF14
:1026E000FD0EDBCFE6FFFE0EDBCFE6FFDADDE552C7
:1026F000E552E552DF6EDF5002E0DF5002D0000EFF
:1027000000D0E552E552E7CFD9FF1200D9CFE6FF5E
:10271000E1CFD9FF030EE126010EDB68020EDB6874
:1027200070DEDF6EDF5002E0DF505DD0FC0EDB506C
:1027300037E0FC0EDB5034E00400FD0EDBCFE9FF98
:10274000FE0EDBCFEAFFEF50E66E07DFE552DF6EED
:10275000DF5003E08EDEDF5046D0FD0EDB2AFE0E9A
:1027600001E3DB2A0001C451C51117E0FC0EDB04B4
:1027700014E0E66A73EC1AF0E552E66A91EC1AF09E
:10278000E552F3CF14F0F4CF15F00001C451145CFE
:10279000C551155802E20400F0D7FC0EDB06C9D77C
:1027A000010EDB68020EDB68040EC7140EE0010E9A
:1027B000DB06DBCF14F0020E01E2DB06DBCF15F007
:1027C0001450151002E00400EFD7D950010FE96E44
:1027D000DACFEAFFEE50ED1003E14BDE0D0E03D031
:1027E00048DE000E00D0D9CFE1FFE552E7CFD9FF98
:1027F0001200D9CFE6FFE1CFD9FFFE0EDB500A0D64
:10280000F3CFC4F0F4CFC5F0E552E7CFD9FF120003
:102810000A0E146E156AC4C006F0C5C007F014C0D5
:102820000BF015C00CF02EEC1DF0065000D012007D
:102830003D3D3D3D3E436865636B73756D2066614C
:10284000696C7572650D0A000D0A203D3D3D3E4ED6
:102850004F2041434B206461746120636F756E6546
:10286000723D3D30000D0A203D3D3D3E416D5553CA
:102870004247656E5478497342757379000D0A3D7D
:102880003D3E204932435F4745545F5350454544E0
:1028900020283078257829726571756573746564B0
:1028A000000D0A3D3D3E204932435F5345545F537E
:1028B0005045454420283078257829726571756522
:1028C00073746564000D0A3D3D3E204932435F53F9
:1028D00045545F44454C4159207265717565737468
:1028E0006564000D0A3D3D3E20494932435F47453E
:1028F000545F44454C415920283078257829726529
:1029000071756573746564000D0A3D3D3E20493262
:10291000435F4745545F535452494E472825642925
:1029200020726571756573746564000D0A3D3D3EE6
:102930002057524954455F535452494E4728256405
:102940002920726571756573746564000D0A3D3DDB
:102950003E204932435F52445F4E4F5F41434B201C
:1029600072657175657374656420283078257829DF
:10297000000D0A3D3D3E204932435F52445F4143D2
:102980004B207265717565737465642028307825F5
:102990007829000D0A3D3D3E2052455045415420C6
:1029A00053415452542072657175657374656400A7
:1029B0000D0A206F7065726174696F6E2051505FEF
:1029C0004932435F5270656174537461727420665A
:1029D00061696C656420000D0A3D3D3E20577269B7
:1029E00074652044617461207265717565737465E6
:1029F00064203078257820535350434F4E323D3079
:102A0000782578206E5374617475733D2578000DB8
:102A10000A2020206F7065726174696F6E20666194
:102A2000696C656420000D0A3D3D3E2053544F50B3
:102A30002062697420726571756573746564000D38
:102A40000A206F7065726174696F6E2051505F4922
:102A500032435F53746F70206661696C6564200057
:102A60000D0A3D3D3E2053746172742062697420EA
:102A7000726571756573746564000D0A206F706509
:102A8000726174696F6E2051505F4932435F5374B5
:102A9000617274206661696C656420000D0A3D3DB9
:102AA0003E2049324320636C6F73652072657175F7
:102AB0006573746564000D0A3D3D3E204932432034
:102AC0006F70656E20726571756573746564000D55
:102AD0000A3D3D3E204745545F5253545F53544195
:102AE0005420726571756573746564000D0A3D3D0F
:102AF0003E2052455345545F5253545F434E542039
:102B000072657175657374656400257820000D0A1F
:102B10003D3E000D0A2A2A2A205553422D493243B0
:102B200020627920512D50726F746F205379737425
:102B3000656D2032303035202A2A2A0D0A000D0A10
:102B40005265736574205374617475733A52434FC0
:102B50004E3D307825780A0004011851600BE84298
:102B6000E842E842E842E842000901E055D0195144
:102B7000070A51E00B0A4FE0070A40E0010A2CE087
:102B80000B0A28E0020A26E0030A22E0080A12E003
:102B9000010A0EE00F0A0AE0030A01E03CD000013E
:102BA000010EAD6F0001040EBC6F36D036D834D0A4
:102BB00090D832D00001010EAD6F0001BE0EAE6F95
:102BC000000EAF6F0001BD930001010EB26F24D063
:102BD000A8D822D0F4D820D00001010EAD6F040196
:102BE0001C510001AE6FAF6BBF0EAE27000EAF23BE
:102BF0000001BD930001010EB26F0ED00001010E65
:102C0000AD6F04011C51EA6ABF0FE96E000EEA22A3
:102C10001AC4EFFF01D000D01200800E0401185D2D
:102C200057E11B51030A34E0010A10E0030A01E0F6
:102C30004DD00001010EAD6F0001380EAE6F370EA2
:102C4000AF6F120E0001B26FB36B40D00001010EE6
:102C5000AD6F04011A51F66EF76AD890F636F73662
:102C6000AA0EF626370EF7220900F5CFAEF00A00BD
:102C7000F5CFAFF0020E0001F76AAE25F66EAF5148
:102C8000F7220900F5CFB2F00A00F5CFB3F01ED05D
:102C90000001010EAD6F04011A51F66EF76AD8906B
:102CA000F636F736AE0EF626370EF7220900F5CFC8
:102CB000AEF00A00F5CFAFF0AEC0F6FFAFC0F7FF41
:102CC0000800F5500001B26FB36B00D00001BD8366
:102CD00012000001010EAD6F0F0EE66E710EE66E72
:102CE0000F0EE66E26EC19F0E552E552E552010EA4
:102CF000E66EBF0EE66E000EE66E26EC19F0E552AB
:102D0000E552E5521AC4BEF004011A5104E1000173
:102D1000050EBC6F05D00001060EBC6FDCEC19F08F
:102D200012000401206B216B040118511F0B020AD1
:102D300014E0030A0EE0010A01E033D00001010EA5
:102D4000AD6F040120810001BDA102D004012083E8
:102D500028D00001010EAD6F24D00001010EAD6F2F
:102D600004011C510F0B080DF350156A000F146E6F
:102D7000040E15221C51800B01E0010E040DF350CE
:102D800000011424B06F000E1520B16FB0C0E9FF30
:102D9000B1C0EAFFEF50040B03E00401010E206F05
:102DA00000D00001AD050AE10001200EAE6F040E57
:102DB000AF6F0001BD930001020EB26F120004015B
:102DC0001A0510E118511F0B00090CE10001010E5A
:102DD000AD6F030E0401195D03E10001BD8102D056
:102DE0000001BD9104011A513AE118511F0B02086C
:102DF00036E11C510F0B000932E00001010EAD6FEE
:102E000004011C510F0B080DF350156A000F146ECE
:102E1000040E15221C51800B01E0010E040DF3502D
:102E200000011424B06F000E1520B16F030E0401D1
:102E3000195D07E1840EB0C0E9FFB1C0EAFFEF6E93
:102E40000ED01CAF06D0B0C0E9FFB1C0EAFFEF6AF8
:102E500006D0880EB0C0E9FFB1C0EAFFEF6E1200E5
:102E60006C5002E0000E01D0010E00090BE00401DD
:102E700000513C0BE842E8420D0802E10CD801D0B9
:102E80001CD808D06C5002E0000E01D0010E0409DD
:102E900001E023D81200D9CFE6FFE1CFD9FFE652F7
:102EA0000001AC6BAD6BB26BB36BACEC15F0D5D86D
:102EB000E552E552E7CFD9FF1200020E0001AC5DEA
:102EC0000AE192D8040100BD03D0C80E006F02D001
:102ED000880E006F01D007D91200040E0001BC5DFE
:102EE0000AE11AC46EFF6E50000803E2050EBC6FC3
:102EF00002D0030EBC6F0001AC050AE10BD804013F
:102F000004BD03D0C80E046F02D0880E046F01D038
:102F1000EAD81200D9CFE6FFE1CFD9FF020EE126B1
:102F20000001080EB25D000EB35905E2B2C0DEFF2B
:102F3000B3C0DDFF03D0080EDE6EDD6A040104932A
:102F40000491010EDB500413DFCF05F4000EDB50BB
:102F50000001B25F010EDB50B35B200EB06F040EB8
:102F6000B16F0001BDA31ED0D9CFE9FFDACFEAFFD0
:102F7000EE50ED1016E0AEC0F6FFAFC0F7FF080050
:102F8000F550B0C0E9FFB1C0EAFFEF6E0001B02B11
:102F9000000EB123AE2BAF23DF06010E01E2DB06EC
:102FA000E3D71CD0D9CFE9FFDACFEAFFEE50ED101E
:102FB00015E0AEC0E9FFAFC0EAFFEF50B0C0E9FFD7
:102FC000B1C0EAFFEF6E0001B02B000EB123AE2BB3
:102FD000AF23DF06010E01E2DB06E4D7D9CFE1FF24
:102FE000E552E7CFD9FF1200D9CFE6FFE1CFD9FFF5
:102FF000020EE126030E04010015E76E010EE7CF75
:10300000DBFF01C4DFFFDE500001B227DD50B32338
:10301000200EAE6F040EAF6FD9CFE9FFDACFEAFF13
:10302000EE50ED1014E0AEC0E9FFAFC0EAFFEF5084
:10303000B0C0E9FFB1C0EAFFEF6EB02B000EB123C4
:10304000AE2BAF23DF06010E01E2DB06E5D7D9CFB9
:10305000E1FFE552E7CFD9FF12000001AD510CE1CD
:103060000401080E016F180E026F040E036F840E28
:10307000006F0401046F35D0040118AF22D00001A5
:10308000B25104011E5D0001B35104011F5904E255
:103090001EC4B2F01FC4B3F03DDF0001010EAC6FDF
:1030A0000401080E016F180E026F040E036F800EEC
:1030B000006F0401200E066F040E076FC80E046F28
:1030C00010D00001020EAC6F0401056BC80E046F36
:1030D0000401080E016F200E026F040E036FC80E6C
:1030E000006F6D9812000001AC6B0401080E016FB7
:1030F000180E026F040E036F880E006F0401046B3C
:1031000012006DA60CD80001BC0508E16DBA06D00E
:10311000686A696A69806988020EBC6F12006D6A0C
:10312000696A6D860001010EBC6F12006D6A696AE2
:103130000001BC6B120096EF18F00001BC5101E1D8
:103140003AD06850040B04E06950040B01E038D811
:103150006DB231D06850010B04E06950010B01E001
:1031600053D86850100B04E06950100B01E024D8CC
:103170006850400B04E06950400B01E03AD86850B9
:10318000200B04E06950200B01E035D86850020B99
:1031900004E06950020B01E035D8030E0001BC5D6C
:1031A00001E209D06850080B06E06950080B03E003
:1031B00030EC17F068961200698468986D821200EE
:1031C0006D926994689412000001BDA111D0F8DFDE
:1031D0006D840001080EC06F070EC16F0001C007AB
:1031E000000EC15B04000001C051C111F7E16D94F4
:1031F0001200689C120070A003D073EC18F070905D
:10320000689A1200689212006A6A686A9F0E6B6E72
:103210007B0E696E6E6A0F0EE66E710EE66E0F0E15
:10322000E66E14D8E552E552E552160E706E68A6A9
:1032300002D06896FCD76D9873EC18F00001BD9130
:103240000001BE6B0001030EBC6F1200D9CFE6FF78
:10325000E1CFD9FFFD0EDBCFE9FFFE0EDBCFEAFFAA
:10326000FC0EDB5005E0EE6AFC0EDB060400F8D72E
:10327000E552E7CFD9FF1200DACFE4FFE2CFDAFF61
:10328000E9CFE4FFEACFE4FFE652D9CFE6FFE1CF92
:10329000D9FFE652F2A416D0F294D768D10ED66EBA
:1032A000DF6A040EDF5C0EE2EA6ADF34FE0BEA3608
:1032B000E96EB40EE926000EEA22EE2A000EEF2295
:1032C000DF2AEFD7E552E552E7CFD9FFE552E5CF48
:1032D000EAFFE5CFE9FFE5CFDAFF1100D0CFCAF072
:1032E0000001C82B4AD80001CA51E66EE66A3E0EBC
:1032F000146E2B0E156E166A14C0E6FF15C0E6FF9D
:1033000016C0E6FF10EC1BF0F56E050EE15EF55001
:103310008A86010EE66E73EC1AF0E552010EE66E37
:1033200091EC1AF0E552F3CF14F0F4CF15F0E80E5B
:10333000145C030E155802E20400F0D78A96010EC1
:10334000E66E73EC1AF0E552010EE66E91EC1AF09F
:10335000E552F3CF14F0F4CF15F0E80E145C030E31
:10336000155802E20400F0D78A866F9E040012D836
:10337000040056EC04F0FAD712000F0EC11292822C
:10338000140E6F6E0001BC6B0001BD6B0001BE6BC3
:103390002EEF04F081EC18F06FBE02D09DEC18F017
:1033A00012000001C85100D012000001CA5100D023
:1033B00012000001C86B12000001C66B1E0E716E78
:1033C0000401400E096F280E0A6F040E0B6F880E61
:1033D000086F0401680E0E6F040E0F6F400E0C6F25
:1033E0001200D9CFE6FFE1CFD9FFE652FC0EDB5049
:1033F000400805E2400EF36EFC0EF3CFDBFFDF6A00
:10340000FC0EDB50DF5C19E2DF50E76EFD0EDBCF18
:10341000E9FFFE0EDBCFEAFFE750E926000EEA22C5
:10342000EF50E66EDF50EA6A680FE96E040EEA229A
:10343000E552E750EF6EDF2AE3D7FC0EDBCF0DF449
:10344000400E04010C170C7D880E0C13E552E5525A
:10345000E7CFD9FF1200D9CFE6FFE1CFD9FF0001B6
:10346000C66B040108BF30D0FC0EDBCF14F009514D
:10347000D880145403E2FC0E09C4DBFF0001C66BC4
:10348000FC0EDB50C65D19E2C651EA6A280FE96EF0
:10349000040EEA22EF50E66EC651E76EFD0EDBCF5A
:1034A000E9FFFE0EDBCFEAFFE750E926000EEA2235
:1034B000E552E750EF6EC62BE3D70401400E096FCB
:1034C0000817087D880E08130001C65100D0E55288
:1034D000E7CFD9FF1200970ED56EF28AF194D08E05
:1034E000F28EF28C1200D9CFE6FFE1CFD9FF040EA5
:1034F000F36EFE0EDBCFF4FFF350F45C0EE2F29EAF
:10350000FE0EEA6ADB34FE0BEA36E96EB40EE926FB
:10351000000EEA22EE6AED6AF28EE552E7CFD9FF9D
:103520001200D9CFE6FFE1CFD9FF020EE126040E4B
:10353000F36EFE0EDBCFF4FFF350F45C19E2F29E63
:10354000FE0EEA6ADB34FE0BEA36E96EB40EE926BB
:10355000000EEA22EECFDEFFEDCFDDFFF28EDECFF2
:1035600014F0DDCF15F014C0F3FF15C0F4FF03D045
:10357000F36AF46A00D0D9CFE1FFE552E7CFD9FF73
:1035800012002A0EF66E080EF76E000EF86E00019D
:103590000900F550A76F0900F550A86F03E1A76770
:1035A00001D03DD00900F550A26F0900F550A36F7E
:1035B0000900F550A46F09000900F550E96E0900F3
:1035C000F550EA6E090009000900F550A56F0900E1
:1035D000F550A66F09000900F6CFA9F0F7CFAAF0C1
:1035E000F8CFABF0A2C0F6FFA3C0F7FFA4C0F8FF6E
:1035F0000001A55302E1A65307E00900F550EE6E65
:10360000A507F8E2A607F9D7A9C0F6FFAAC0F7FFF9
:10361000ABC0F8FF0001A707000EA85BBFD71200E0
:10362000D9CFE6FFDACFE6FFE1CFD9FFE2CFDAFF6D
:10363000E652E652E652E652D950FB0F146EFF0EE8
:10364000DA20156E14C0DEFFDD6EDECFE6FFDDCFC3
:10365000E6FFFB0EDBCFE6FFFC0EDBCFE6FFFD0E49
:10366000DBCFE6FFC2C0E6FFC3C0E6FFCCEC0AF04A
:10367000F56E070EE15C02E2E16AE552E16EF5509B
:10368000020EF3CFDBFF030EF4CFDBFF020EDBCF26
:1036900014F0030EDBCF15F014C0F3FF15C0F4FFD8
:1036A000D9CFE1FFDACFE2FFE552E5CFDAFFE7CF8E
:1036B000D9FF1200D9CFE6FFDACFE6FFE1CFD9FF7D
:1036C000E2CFDAFFFB0EDBCF14F0FC0EDBCF15F000
:1036D0000001800E15141AE1FB0EDBCFE9FFFC0E92
:1036E000DBCFEAFFEECFF3FFEDCFF4FFEE2A000EC3
:1036F000EF22F3CFE9FFF4CFEAFFFD0EDBCFEFFFC0
:10370000EF50156AF36E15C0F4FF10D0FB0EDB50BE
:10371000FE0806E1FD0EDBCFE6FF56EC1DF005D0FE
:10372000FD0EDBCFE6FF79EC1DF0E552E552E5CF6B
:10373000DAFFE7CFD9FF12001201000200000008F3
:10374000D8040B0000000102000109022000010161
:103750000080FA09040000020000000007050103D0
:1037600040002007058103400020040309042003D2
:1037700051002D00500072006F0074006F00200097
:10378000530079007300740065006D002E001C0367
:1037900051004200720069006400670065002D005E
:1037A0004900320043002D0055004A374A376A3736
:1037B0006E378E3704500902F3CF00F0F4CF01F0DA
:1037C0000A02F3500126000EF420026E04500B0290
:1037D000F3500226000EF420036E04500C02F35046
:1037E000032605500902F3500126F4500222000E70
:1037F000032205500A02F3500226F450032205501A
:103800000B02F350032606500902F3500226F4502F
:10381000032206500A02F350032607500902F35010
:1038200003261200D9CFE6FFDACFE6FFE1CFD9FFBA
:10383000E2CFDAFFAC6AAB6AFD0EDBB0AC88DBA28C
:1038400002D0AC8CAB8CDBB4AC8EDBA602D0AB88E8
:1038500001D0AB8ADBA802D0AC8401D0AC949E9896
:10386000DBAC02D09D8A01D09D9A9E9ADBAE02D03D
:103870009D8801D09D98FB0EDB50AF6EAC8AAB8E5D
:10388000E552E5CFDAFFE7CFD9FF1200FE0EE3CF16
:10389000E9FFFF0EE3CFEAFFF36AF46AEE5203E0BA
:1038A000F34AF42AFBD71200FF0EE3CFF8FFE552EC
:1038B000FF0EE3CFF7FFE552FF0EE3CFF6FFE55231
:1038C000E66AE66AE66A0900F55209E0FD0EE32AB7
:1038D00005E1FE0EE32A02E1FF0EE32AF4D7FD0E16
:1038E000E3CF05F0FE0EE3CF06F0FF0EE3CF07F0C7
:1038F0001200D9CFE6FFDACFE6FFE1CFD9FFE2CF62
:10390000DAFFACA2FED7FB0EDBCFF6FFFC0EDBCF5F
:10391000F7FFFD0EDBCFF8FF0800F550E66E17EC61
:103920001DF0E552D950FB0FE96EFF0EDA20EA6E6A
:10393000EFCFF6FFEE2AEFCFF7FF000EEE22EFCF2C
:10394000F8FFEE220800F550DCE1E552E5CFDAFFA2
:10395000E7CFD9FF120007C013F006C012F00650DF
:103960000B02F4CF05F0F3CF04F007500C02F4CFB4
:1039700007F0F3CF06F00B02F3500526F4500622B1
:10398000E86A072212500C02F3500526F450062272
:10399000E86A07220CAED1EF1CF01250065E1350FD
:1039A000075A13AE000C0B50065E0C50075A000C61
:1039B000036A026A016A006A200EE76ED890043634
:1039C000053606360736003601360236033609500C
:1039D000005C0A5001580B5002580C50035809E380
:1039E0000950005E0A50015A0B50025A0C50035AFB
:1039F000042AE72EE4D71200D9CFE6FFDACFE6FF9C
:103A0000E1CFD9FFE2CFDAFF3F0EC716C66AC56A1B
:103A1000FD0EDB50C612FC0EDB50C7129382938062
:103A2000C68AE552E5CFDAFFE7CFD9FF1200D9CF3A
:103A3000E6FFDACFE6FFE1CFD9FFE2CFDAFFACACA9
:103A400004D0AC900001C7B3AC80FD0EDB50AD6E6E
:103A5000E552E5CFDAFFE7CFD9FF1200036A026A29
:103A6000100EE76ED89006360736023603360B5036
:103A7000025C0C50035805E30B50025E0C50035AD5
:103A8000062AE72EF0D71200F36AF46AFF0EE1244B
:103A9000E96EFF0EE220EA6EED6607D02F0EEF64AE
:103AA00004D03A0EEF6001D0F32A1200FF0EE3506B
:103AB000ACBA04D0AF6AAB8EAC8A949CACA2FED7F1
:103AC000AD6EF36EF46A120013EE00F023EE00F018
:103AD000F86A0F9CC1EC1AF06EEC19F0FDD71200D9
:103AE0003031323334353637383961626364656674
:103AF00000001200FEFF000000FFFFFFFFFFFFFFBE
:103B0000FFFFFFFFFFFFFFFFFFFFFFFFFFFFFFFFC5
:103B1000FFFFFFFFFFFFFFFFFFFFFFFFFFFFFFFFB5
:103B2000FFFFFFFFFFFFFFFFFFFFFFFFFFFFFFFFA5
:103B3000FFFFFFFFFFFFFFFFFFFFFFFFFFFFFFFF95
:0200000400F00A
:00000001FF
